******************************************************************************
                  TI ARM Linker PC v18.1.2                     
******************************************************************************
>> Linked Tue Feb 12 12:29:39 2019

OUTPUT FILE NAME:   <Memory_board.out>
ENTRY POINT SYMBOL: "_c_int00_noargs"  address: 00000e15


MEMORY CONFIGURATION

         name            origin    length      used     unused   attr    fill
----------------------  --------  ---------  --------  --------  ----  --------
  FLASH                 00000000   00100000  000010bc  000fef44  R  X
  SRAM                  20000000   00040000  00010028  0002ffd8  RW X


SEGMENT ALLOCATION MAP

run origin  load origin   length   init length attrs members
----------  ----------- ---------- ----------- ----- -------
00000000    00000000    000010c0   000010c0    r-x
  00000000    00000000    0000026c   0000026c    r-- .intvecs
  0000026c    0000026c    00000d68   00000d68    r-x .text
  00000fd4    00000fd4    000000b0   000000b0    r-- .const
  00001088    00001088    00000038   00000038    r-- .cinit
20000000    20000000    00010028   00000000    rw-
  20000000    20000000    0000c010   00000000    rw- .bss
  2000c010    2000c010    00004000   00000000    rw- .stack
  20010010    20010010    00000018   00000000    rw- .data


SECTION ALLOCATION MAP

 output                                  attributes/
section   page    origin      length       input sections
--------  ----  ----------  ----------   ----------------
.intvecs   0    00000000    0000026c     
                  00000000    0000026c     tm4c123gh6pm_startup_ccs.obj (.intvecs)

.text      0    0000026c    00000d68     
                  0000026c    00000374     TM4C129_SSI3_MacronixFlash.obj (.text:main)
                  000005e0    000001ea     uartstdio.obj (.text:UARTvprintf)
                  000007ca    00000132     driverlib.lib : gpio.obj (.text:GPIOPadConfigSet)
                  000008fc    0000009c     rtsv7M4_T_le_v4SPD16_eabi.lib : memcpy_t2.asm.obj (.text)
                  00000998    00000090     TM4C129_SSI3_MacronixFlash.obj (.text:SSILibSendEraseCommand)
                  00000a28    0000007a     rtsv7M4_T_le_v4SPD16_eabi.lib : memset_t2.asm.obj (.text)
                  00000aa2    00000002     tm4c123gh6pm_startup_ccs.obj (.text:FaultISR)
                  00000aa4    00000074     TM4C129_SSI3_MacronixFlash.obj (.text:SSILibSendReadIDAdvMode)
                  00000b18    00000068     rtsv7M4_T_le_v4SPD16_eabi.lib : copy_decompress_lzss.c.obj (.text:decompress:lzss:__TI_decompress_lzss)
                  00000b80    00000060     uartstdio.obj (.text:UARTStdioConfig)
                  00000be0    0000004c     TM4C129_SSI3_MacronixFlash.obj (.text:InitConsole)
                  00000c2c    0000004c     TM4C129_SSI3_MacronixFlash.obj (.text:SSILibSendReadDataAdvBi)
                  00000c78    0000004c     TM4C129_SSI3_MacronixFlash.obj (.text:SSILibSendReadStatusRegister)
                  00000cc4    00000048     driverlib.lib : gpio.obj (.text:GPIOPinConfigure)
                  00000d0c    00000048     uartstdio.obj (.text:UARTwrite)
                  00000d54    00000044     rtsv7M4_T_le_v4SPD16_eabi.lib : autoinit.c.obj (.text:__TI_auto_init_nobinit_nopinit:__TI_auto_init_nobinit_nopinit)
                  00000d98    00000040                                   : u_divt2.asm.obj (.text)
                  00000dd8    0000003c     driverlib.lib : ssi.obj (.text:SSIConfigSetExpClk)
                  00000e14    00000038     rtsv7M4_T_le_v4SPD16_eabi.lib : boot_cortex_m.c.obj (.text:_c_int00_noargs:_c_int00_noargs)
                  00000e4c    00000034     driverlib.lib : sysctl.obj (.text:SysCtlPeripheralEnable)
                  00000e80    00000034     rtsv7M4_T_le_v4SPD16_eabi.lib : rand.c.obj (.text:rand)
                  00000eb4    0000002a     driverlib.lib : gpio.obj (.text:GPIODirModeSet)
                  00000ede    0000001a     TM4C129_SSI3_MacronixFlash.obj (.text:SSILibDeviceBusyCheck)
                  00000ef8    0000001a     uartstdio.obj (.text:UARTprintf)
                  00000f12    00000012     driverlib.lib : gpio.obj (.text:GPIOPinTypeSSI)
                  00000f24    00000012                   : gpio.obj (.text:GPIOPinTypeUART)
                  00000f36    00000012                   : ssi.obj (.text:SSIAdvDataPutFrameEnd)
                  00000f48    00000012                   : ssi.obj (.text:SSIDataGetNonBlocking)
                  00000f5a    0000000e     rtsv7M4_T_le_v4SPD16_eabi.lib : copy_decompress_none.c.obj (.text:decompress:none:__TI_decompress_none)
                  00000f68    0000000c     driverlib.lib : ssi.obj (.text:SSIAdvModeSet)
                  00000f74    0000000c                   : ssi.obj (.text:SSIDataGet)
                  00000f80    0000000c     rtsv7M4_T_le_v4SPD16_eabi.lib : copy_zero_init.c.obj (.text:decompress:ZI:__TI_zero_init)
                  00000f8c    0000000a     driverlib.lib : ssi.obj (.text:SSIAdvFrameHoldEnable)
                  00000f96    0000000a                   : ssi.obj (.text:SSIDataPut)
                  00000fa0    0000000a                   : ssi.obj (.text:SSIEnable)
                  00000faa    00000008                   : ssi.obj (.text:SSIBusy)
                  00000fb2    00000006     tm4c123gh6pm_startup_ccs.obj (.text:ResetISR)
                  00000fb8    00000006     driverlib.lib : sysctl.obj (.text:SysCtlDelay)
                  00000fbe    00000006                   : uart.obj (.text:UARTClockSourceSet)
                  00000fc4    00000004     rtsv7M4_T_le_v4SPD16_eabi.lib : pre_init.c.obj (.text:_system_pre_init)
                  00000fc8    00000004                                   : exit.c.obj (.text:abort:abort)
                  00000fcc    00000002     tm4c123gh6pm_startup_ccs.obj (.text:IntDefaultHandler)
                  00000fce    00000002     tm4c123gh6pm_startup_ccs.obj (.text:NmiSR)
                  00000fd0    00000002     rtsv7M4_T_le_v4SPD16_eabi.lib : _lock.c.obj (.text:_nop)
                  00000fd2    00000002                                   : div0.asm.obj (.text)

.const     0    00000fd4    000000b0     
                  00000fd4    00000090     driverlib.lib : gpio.obj (.const:g_pui32GPIOBaseAddrs)
                  00001064    0000000c     uartstdio.obj (.const:g_ui32UARTBase)
                  00001070    0000000c     uartstdio.obj (.const:g_ui32UARTPeriph)
                  0000107c    00000008     TM4C129_SSI3_MacronixFlash.obj (.const:$P$T0$1)

.cinit     0    00001088    00000038     
                  00001088    00000013     (.cinit..data.load) [load image, compression = lzss]
                  0000109b    00000001     --HOLE-- [fill = 0]
                  0000109c    0000000c     (__TI_handler_table)
                  000010a8    00000008     (.cinit..bss.load) [load image, compression = zero_init]
                  000010b0    00000010     (__TI_cinit_table)

.init_array 
*          0    00000000    00000000     UNINITIALIZED

.bss       0    20000000    0000c010     UNINITIALIZED
                  20000000    00002000     (.common:pui32DataRx1)
                  20002000    00002000     (.common:pui32DataRx2)
                  20004000    00002000     (.common:pui32DataRx3)
                  20006000    00002000     (.common:pui32DataTx1)
                  20008000    00002000     (.common:pui32DataTx2)
                  2000a000    00002000     (.common:pui32DataTx3)
                  2000c000    00000004     (.common:pui32Dummy)
                  2000c004    00000004     (.common:ui32DeviceID)
                  2000c008    00000004     (.common:ui32Index)
                  2000c00c    00000004     (.common:ui32SysClockFreq)

.data      0    20010010    00000018     UNINITIALIZED
                  20010010    00000008     rtsv7M4_T_le_v4SPD16_eabi.lib : _lock.c.obj (.data:$O1$$)
                  20010018    00000005     uartstdio.obj (.data)
                  2001001d    00000004     TM4C129_SSI3_MacronixFlash.obj (.data:g_ui8InstrReadID)
                  20010021    00000003     --HOLE--
                  20010024    00000004     rtsv7M4_T_le_v4SPD16_eabi.lib : rand.c.obj (.data)

.stack     0    2000c010    00004000     UNINITIALIZED
                  2000c010    00000004     rtsv7M4_T_le_v4SPD16_eabi.lib : boot_cortex_m.c.obj (.stack)
                  2000c014    00003ffc     --HOLE--

MODULE SUMMARY

       Module                           code   ro data   rw data
       ------                           ----   -------   -------
    .\
       TM4C129_SSI3_MacronixFlash.obj   1398   8         49172  
       uartstdio.obj                    684    24        5      
       tm4c123gh6pm_startup_ccs.obj     12     620       0      
    +--+--------------------------------+------+---------+---------+
       Total:                           2094   652       49177  
                                                                
    C:/ti/TivaWare_C_Series-2.1.4.178--new/driverlib/ccs/Debug/driverlib.lib
       gpio.obj                         456    144       0      
       ssi.obj                          158    0         0      
       sysctl.obj                       58     0         0      
       uart.obj                         6      0         0      
    +--+--------------------------------+------+---------+---------+
       Total:                           678    144       0      
                                                                
    C:\ti\ccsv8\tools\compiler\ti-cgt-arm_18.1.2.LTS\lib\rtsv7M4_T_le_v4SPD16_eabi.lib
       memcpy_t2.asm.obj                156    0         0      
       memset_t2.asm.obj                122    0         0      
       copy_decompress_lzss.c.obj       104    0         0      
       autoinit.c.obj                   68     0         0      
       u_divt2.asm.obj                  64     0         0      
       boot_cortex_m.c.obj              56     0         0      
       rand.c.obj                       52     0         4      
       copy_decompress_none.c.obj       14     0         0      
       copy_zero_init.c.obj             12     0         0      
       _lock.c.obj                      2      0         8      
       exit.c.obj                       4      0         0      
       pre_init.c.obj                   4      0         0      
       div0.asm.obj                     2      0         0      
    +--+--------------------------------+------+---------+---------+
       Total:                           660    0         12     
                                                                
       Stack:                           0      0         16384  
       Linker Generated:                0      55        0      
    +--+--------------------------------+------+---------+---------+
       Grand Total:                     3432   851       65573  


LINKER GENERATED COPY TABLES

__TI_cinit_table @ 000010b0 records: 2, size/record: 8, table size: 16
	.data: load addr=00001088, load size=00000013 bytes, run addr=20010010, run size=00000018 bytes, compression=lzss
	.bss: load addr=000010a8, load size=00000008 bytes, run addr=20000000, run size=0000c010 bytes, compression=zero_init


LINKER GENERATED HANDLER TABLE

__TI_handler_table @ 0000109c records: 3, size/record: 4, table size: 12
	index: 0, handler: __TI_decompress_lzss
	index: 1, handler: __TI_decompress_none
	index: 2, handler: __TI_zero_init


GLOBAL SYMBOLS: SORTED ALPHABETICALLY BY Name 

address   name                          
-------   ----                          
00000fc9  C$$EXIT                       
00000eb5  GPIODirModeSet                
000007cb  GPIOPadConfigSet              
00000cc5  GPIOPinConfigure              
00000f13  GPIOPinTypeSSI                
00000f25  GPIOPinTypeUART               
00000be1  InitConsole                   
00000fb3  ResetISR                      
00000f37  SSIAdvDataPutFrameEnd         
00000f8d  SSIAdvFrameHoldEnable         
00000f69  SSIAdvModeSet                 
00000fab  SSIBusy                       
00000dd9  SSIConfigSetExpClk            
00000f75  SSIDataGet                    
00000f49  SSIDataGetNonBlocking         
00000f97  SSIDataPut                    
00000fa1  SSIEnable                     
00000edf  SSILibDeviceBusyCheck         
00000999  SSILibSendEraseCommand        
00000c2d  SSILibSendReadDataAdvBi       
00000aa5  SSILibSendReadIDAdvMode       
00000c79  SSILibSendReadStatusRegister  
00000fb9  SysCtlDelay                   
00000e4d  SysCtlPeripheralEnable        
00000fbf  UARTClockSourceSet            
00000b81  UARTStdioConfig               
00000ef9  UARTprintf                    
000005e1  UARTvprintf                   
00000d0d  UARTwrite                     
20010010  __STACK_END                   
00004000  __STACK_SIZE                  
2000c110  __STACK_TOP                   
000010b0  __TI_CINIT_Base               
000010c0  __TI_CINIT_Limit              
0000109c  __TI_Handler_Table_Base       
000010a8  __TI_Handler_Table_Limit      
00000d55  __TI_auto_init_nobinit_nopinit
00000b19  __TI_decompress_lzss          
00000f5b  __TI_decompress_none          
ffffffff  __TI_pprof_out_hndl           
ffffffff  __TI_prof_data_size           
ffffffff  __TI_prof_data_start          
00000000  __TI_static_base__            
00000f81  __TI_zero_init                
00000fd3  __aeabi_idiv0                 
00000fd3  __aeabi_ldiv0                 
00000a29  __aeabi_memclr                
00000a29  __aeabi_memclr4               
00000a29  __aeabi_memclr8               
000008fd  __aeabi_memcpy                
000008fd  __aeabi_memcpy4               
000008fd  __aeabi_memcpy8               
00000a2b  __aeabi_memset                
00000a2b  __aeabi_memset4               
00000a2b  __aeabi_memset8               
00000d99  __aeabi_uidiv                 
00000d99  __aeabi_uidivmod              
ffffffff  __binit__                     
ffffffff  __c_args__                    
UNDEFED   __mpu_init                    
2000c010  __stack                       
00000e15  _c_int00_noargs               
20010010  _lock                         
00000fd1  _nop                          
UNDEFED   _system_post_cinit            
00000fc5  _system_pre_init              
20010014  _unlock                       
00000fc9  abort                         
ffffffff  binit                         
00000000  g_pfnVectors                  
2001001d  g_ui8InstrReadID              
0000026d  main                          
000008fd  memcpy                        
00000a31  memset                        
20000000  pui32DataRx1                  
20002000  pui32DataRx2                  
20004000  pui32DataRx3                  
20006000  pui32DataTx1                  
20008000  pui32DataTx2                  
2000a000  pui32DataTx3                  
2000c000  pui32Dummy                    
00000e81  rand                          
2000c004  ui32DeviceID                  
2000c008  ui32Index                     
2000c00c  ui32SysClockFreq              


GLOBAL SYMBOLS: SORTED BY Symbol Address 

address   name                          
-------   ----                          
00000000  __TI_static_base__            
00000000  g_pfnVectors                  
0000026d  main                          
000005e1  UARTvprintf                   
000007cb  GPIOPadConfigSet              
000008fd  __aeabi_memcpy                
000008fd  __aeabi_memcpy4               
000008fd  __aeabi_memcpy8               
000008fd  memcpy                        
00000999  SSILibSendEraseCommand        
00000a29  __aeabi_memclr                
00000a29  __aeabi_memclr4               
00000a29  __aeabi_memclr8               
00000a2b  __aeabi_memset                
00000a2b  __aeabi_memset4               
00000a2b  __aeabi_memset8               
00000a31  memset                        
00000aa5  SSILibSendReadIDAdvMode       
00000b19  __TI_decompress_lzss          
00000b81  UARTStdioConfig               
00000be1  InitConsole                   
00000c2d  SSILibSendReadDataAdvBi       
00000c79  SSILibSendReadStatusRegister  
00000cc5  GPIOPinConfigure              
00000d0d  UARTwrite                     
00000d55  __TI_auto_init_nobinit_nopinit
00000d99  __aeabi_uidiv                 
00000d99  __aeabi_uidivmod              
00000dd9  SSIConfigSetExpClk            
00000e15  _c_int00_noargs               
00000e4d  SysCtlPeripheralEnable        
00000e81  rand                          
00000eb5  GPIODirModeSet                
00000edf  SSILibDeviceBusyCheck         
00000ef9  UARTprintf                    
00000f13  GPIOPinTypeSSI                
00000f25  GPIOPinTypeUART               
00000f37  SSIAdvDataPutFrameEnd         
00000f49  SSIDataGetNonBlocking         
00000f5b  __TI_decompress_none          
00000f69  SSIAdvModeSet                 
00000f75  SSIDataGet                    
00000f81  __TI_zero_init                
00000f8d  SSIAdvFrameHoldEnable         
00000f97  SSIDataPut                    
00000fa1  SSIEnable                     
00000fab  SSIBusy                       
00000fb3  ResetISR                      
00000fb9  SysCtlDelay                   
00000fbf  UARTClockSourceSet            
00000fc5  _system_pre_init              
00000fc9  C$$EXIT                       
00000fc9  abort                         
00000fd1  _nop                          
00000fd3  __aeabi_idiv0                 
00000fd3  __aeabi_ldiv0                 
0000109c  __TI_Handler_Table_Base       
000010a8  __TI_Handler_Table_Limit      
000010b0  __TI_CINIT_Base               
000010c0  __TI_CINIT_Limit              
00004000  __STACK_SIZE                  
20000000  pui32DataRx1                  
20002000  pui32DataRx2                  
20004000  pui32DataRx3                  
20006000  pui32DataTx1                  
20008000  pui32DataTx2                  
2000a000  pui32DataTx3                  
2000c000  pui32Dummy                    
2000c004  ui32DeviceID                  
2000c008  ui32Index                     
2000c00c  ui32SysClockFreq              
2000c010  __stack                       
2000c110  __STACK_TOP                   
20010010  __STACK_END                   
20010010  _lock                         
20010014  _unlock                       
2001001d  g_ui8InstrReadID              
ffffffff  __TI_pprof_out_hndl           
ffffffff  __TI_prof_data_size           
ffffffff  __TI_prof_data_start          
ffffffff  __binit__                     
ffffffff  __c_args__                    
ffffffff  binit                         
UNDEFED   __mpu_init                    
UNDEFED   _system_post_cinit            

[85 symbols]
